:020000040800F2
:1000000000500020750E0008C90D0008CD0D000835
:10001000D10D0008D50D0008D90D00080000000022
:10002000000000000000000000000000DD0D0008DE
:10003000E10D000800000000E50D0008E90D0008D2
:10004000BD0E0008BD0E0008BD0E0008BD0E000864
:10005000BD0E0008BD0E0008BD0E0008BD0E000854
:10006000BD0E0008BD0E0008BD0E0008BD0E000844
:10007000BD0E0008ED0D0008F90D0008BD0E0008CA
:10008000BD0E0008BD0E0008BD0E0008BD0E000824
:10009000BD0E0008BD0E0008BD0E0008BD0E000814
:1000A000BD0E0008BD0E0008BD0E0008BD0E000804
:1000B000BD0E0008BD0E0008BD0E0008BD0E0008F4
:1000C000BD0E0008BD0E0008BD0E0008BD0E0008E4
:1000D000050E0008BD0E0008BD0E0008BD0E00088C
:1000E000110E0008BD0E0008BD0E00080000000043
:1000F0000000000000000000000000000000000000
:0C01000000000000000000005FF808F1A3
:10010C0010B5054C237833B9044B13B10448AFF345
:10011C0000800123237010BD180000200000000097
:10012C00F425000808B5034B1BB103490348AFF392
:10013C00008008BD000000001C000020F425000811
:10014C0008B500F021FA012000F05AFA00F024FA68
:10015C00322000F055FA00F0F7F900F005FAFD2016
:10016C0000F022FA00F0F8F900F0EEF900F004FAD1
:10017C00122000F019FA00F0EFF900F0E5F900F0A8
:10018C00F3F9AE2000F010FA00F0E6F900F0DCF91B
:10019C0000F0EAF9B32000F007FA00F0DDF900F006
:1001AC00D3F900F0E9F9912000F0FEF900F0D4F950
:1001BC0000F0CAF900F0D8F9CA2000F0F5F900F007
:1001CC00CBF900F0C1F900F0D7F93F2000F0ECF9C1
:1001DC0000F0C2F900F0B8F900F0C6F9A22000F066
:1001EC00E3F900F0B9F900F0AFF900F0C5F900201F
:1001FC0000F0DAF900F0B0F900F0A6F900F0B4F96B
:10020C00A12000F0D1F900F0A7F900F09DF900F061
:10021C00B3F9002000F0C8F900F09EF900F094F951
:10022C0000F0A2F9A02000F0BFF900F095F900F061
:10023C008BF900F0A1F9142000F0B6F900F08CF95C
:10024C0000F082F900F098F9112000F0ADF900F0FF
:10025C0083F900F079F900F087F9B52000F0A4F9E2
:10026C0000F07AF900F070F900F086F9002000F047
:10027C009BF900F071F900F067F900F075F9AB200B
:10028C0000F092F900F068F900F05EF900F074F9F2
:10029C00012000F089F900F05FF900F055F900F049
:1002AC0063F9B42000F080F900F056F900F04CF935
:1002BC0000F062F9A02000F077F900F04DF900F0A1
:1002CC0043F900F059F9FD2000F06EF900F044F903
:1002DC0000F03AF900F048F9C12000F065F900F09F
:1002EC003BF900F031F900F047F9FF2000F05CF920
:1002FC0000F032F900F028F900F036F9C72000F0D0
:10030C0053F900F029F900F01FF900F035F90F202E
:10031C0000F04AF900F020F900F016F900F024F989
:10032C00B92000F041F900F017F900F00DF900F0D8
:10033C001BF9B12000F038F900F00EF900F004F9C7
:10034C0000F01AF9E22000F02FF900F005F900F0A6
:10035C00FBF800F009F9D12000F026F900F0FCF8C8
:10036C0000F0F2F800F008F9822000F01DF900F01E
:10037C00F3F800F0E9F800F0FFF8202000F014F991
:10038C0000F0EAF800F0E0F800F0EEF8BB2000F026
:10039C000BF900F0E1F800F0D7F800F0EDF81F20B1
:1003AC0000F002F900F0D8F800F0CEF800F0DCF81C
:1003BC00B62000F0F9F800F0CFF800F0C5F800F026
:1003CC00DBF8082000F0F0F800F0C6F800F0BCF8FC
:1003DC0000F0CAF8BE2000F0E7F800F0BDF800F01D
:1003EC00B3F800F0C9F8072000F0DEF800F0B4F81C
:1003FC0000F0AAF800F0B8F8A62000F0D5F800F04C
:10040C00ABF800F0A1F800F0AFF8A92000F0CCF8A0
:10041C0000F0A2F80A2000F0F3F800F095F800F0D4
:10042C00A3F8AF2000F0C0F800F096F8BDE8084043
:10043C00322000F0E5B800BFF8B505460C4617466B
:10044C001E461C3500F080F800F08EF8152000F0E8
:10045C00ABF81C3400F080F800F076F800F08CF863
:10046C00E8B200F0A1F800F077F800F06DF800F0B9
:10047C0083F8E0B200F098F800F06EF800F064F841
:10048C0000F072F8752000F08FF800F065F800F0BD
:10049C005BF800F071F8384600F086F800F05CF874
:1004AC0000F052F800F068F8304600F07DF8BDE836
:1004BC00F84000F051B800BF38B50D46044600F0C6
:1004CC0043F800F051F85C2000F06EF800F044F8AE
:1004DC0000F03AF800F050F82946204600F07CF87D
:1004EC00BDE8384000F038B8024A034B1080198040
:1004FC00704700BF0200002000000020064A074B96
:10050C0012881B8841EA011103FB02F25210C9B296
:10051C0001D002F03DB8704700000020020000201E
:10052C0070B516460C46002205463F21104604EBDA
:10053C00C6147F23FFF780FF28194FF40051BDE844
:10054C007040FFF7B9BF00BF00221021014801F035
:10055C000BB800BF0008014001221021014801F036
:10056C0003B800BF0008014000220421014800F03C
:10057C00FBBF00BF0008014001220421014800F02C
:10058C00F3BF00BF0008014000220821014800F021
:10059C00EBBF00BF0008014001220821014800F018
:1005AC00E3BF00BF000801408446002310B5084C8F
:1005BC0082B0012207480DF107018DF807C02370A6
:1005CC0001F000FC2378002BFCD002B010BD00BF62
:1005DC00040000202823002084460A46002310B57E
:1005EC00054C6146054892B2237001F0EBFB237871
:1005FC00002BFCD010BD00BF0400002028230020DD
:10060C0000F0A0BC00220F4B00B5596983B041F03B
:10061C00010159615B69114603F0010301930D203F
:10062C00019B00F0B3FC0D2000F0EEFC00220E202C
:10063C00114600F0ABFC0E2003B05DF804EB00F0AB
:10064C00E3BC00BF00100240F0B5002489B0CDE936
:10065C000444CDE906442E4B2E4F9A692E4E42F09F
:10066C0010029A619A69384602F010020092009AC0
:10067C009A694FF4005142F020029A619A6901255F
:10068C0002F020020192019A9A6942F004029A61E6
:10069C009A6902F004020292029A9A6942F00802E4
:1006AC009A619B69224603F008030393039B00F0B5
:1006BC005BFF224630461C2100F056FF4FF40053DE
:1006CC0004930223384604A90793CDE9055400F09E
:1006DC003DFE1C220323304604A904920793059582
:1006EC00069400F033FE4FF400620C4B04A90C4846
:1006FC00CDE90423069400F029FE22462146282049
:10070C0000F044FC282000F07FFC09B0F0BD00BFD5
:10071C0000100240001001400008014000001110C0
:10072C00000C01400122014B1A707047040000209C
:10073C002DE9F04F0026DFF8BCB183B0DFF8B881AB
:10074C00DFF8B8A1CDF804B0B01C731C18F8062063
:10075C0018F8033018F80050F11C18F8010029099A
:10076C0001F0080141EA0311C9B24F00491007F02A
:10077C00A00701F0550139438F10890007F03307AA
:10078C0001F0C0013943019F5B0817F8019F341D2C
:10079C0003F078030197870818F8044043EAC21362
:1007AC004FEAD20EDFF858B1920007F0380747EA4B
:1007BC00851702F0F802C5F380150EF0180EC9EB80
:1007CC00C90CDBB24EEA441E0BF809504FEA420941
:1007DC0052105FFA8EFE5D0002F055025B1009F0BC
:1007EC00A00949EA020904F0F8044FEA4E0203F0AA
:1007FC0055034FEA6E0EC00005F0A0051D43C0B2B4
:10080C000EF0550302F0A00E620064104EEA030EC7
:10081C0004F0550302F0A0044200401000F0550013
:10082C0002F0A0020243C7F346007F001C4300F015
:10083C00550007F0A0030343A810AD0000F03300EF
:10084C0005F0C00505434FEAA9004FEA890900F0FD
:10085C00330009F0C00949EA00094FEAAE004FEA3B
:10086C008E0E00F033000EF0C00E4EEA000EA010FB
:10087C00A40000F0330004F0C00404439010920074
:10088C0000F0330002F0C002024398109B0000F00D
:10089C00330003F0C0030343080140EA11110AF8C6
:1008AC000C102901D44441EA15118CF801102101D6
:1008BC0041EA141405364FEA09154FEA0E171001D8
:1008CC00190145EA191547EA1E1740EA121241EAC6
:1008DC001313EB2E8CF802508CF803708CF8044038
:1008EC008CF805208CF806307FF42EAF03B0BDE8F1
:1008FC00F08F00BF0B260008B40100203800002048
:10090C00840100200023012230B5012091B04FF466
:10091C0080310224CDE90B33CDE90233CDE9043328
:10092C00089301930A9209934FF480324FF4E01329
:10093C00CDE9060106A8CDE90E230D9400F030FE9A
:10094C0008B172B6FEE703460F254FF480622146CC
:10095C0001A80294039305930195049201F010F8F9
:10096C0008B172B6FEE711B030BD00BF2DE9F04FF3
:10097C0085B000F0C3FAFFF7C5FFFFF765FEFFF780
:10098C0041FE00F01FF900F041F9FFF7D9FB0122FD
:10099C007F4B40214FF48070DFF8F8B17E4CDFF8CC
:1009AC00FCA11A70FFF7A0FD7D4EFFF7C1FE0021E0
:1009BC007C48FFF7A3FD4FF4D068B446DFF8E8E1BC
:1009CC0073460027AEF18000AEF58071AEF5C072B3
:1009DC001CF80750073705EB85050BEB05091BF8D1
:1009EC0005507E2F9D7085708D70957099F8015013
:1009FC0003F1070303F8045CC570CD70D57099F84A
:100A0C00025000F1070003F8035C00F8035C0D7161
:100A1C00157199F8035099F8049003F8025C01F1F0
:100A2C00070100F8025C02F1070201F8025C02F80F
:100A3C00025C03F8019C00F8019C01F8019C02F88F
:100A4C00019CC5D108F52078B8F5C05F0EF5207E65
:100A5C000CF1010CB4D14FF4CC5EDFF850C1304630
:100A6C00ACF17403ACF1F40190F87E20043302EB8A
:100A7C004202A718A25C7D78DA70CA71BA781D712F
:100A8C000D725A7163454A7200F1070001F10401BD
:100A9C00EAD10EF5807EBEF5025F06F1010603F584
:100AAC00807CDCD1DFF808E1424BDFF80CC105E0BB
:100ABC00F24503F107030CF1070C5DD01EF8012F72
:100ACC00002AF5D093F884201F680192D3F80021F6
:100ADC001E79039293F804215D799879D3F88010EC
:100AEC0093F8868093F885900292CCF800708CF87D
:100AFC000460019A93F8066193F805718CF805501F
:100B0C008CF80600D3F8805193F88401CCF880104F
:100B1C008CF8842093F8851193F886218CF88680C4
:100B2C00DDF80C808CF88590CCF80081DDF808801D
:100B3C00F2458CF804818CF805718CF80661CCF8C0
:100B4C0080518CF884018CF885118CF88621D3F8AF
:100B5C00005293F8040293F8051293F806220CF154
:100B6C00070CCCF8F9518CF8FD018CF8FE118CF8BF
:100B7C00FF2103F10703A1D100220A481146FFF718
:100B8C00CFFC4FF400510D4800F0F2FC0CE700BF15
:100B9C0034000020BC2800085C29000895010020C6
:100BAC0038000020A002002020090020941C002006
:100BBC00830100203D260008A10200200010014006
:100BCC0072B6FEE738B5022100234FF400720124FF
:100BDC000C484FF48275C0E90331C0E9054210217D
:100BEC000A22C0E90153C0E908338362064BC16194
:100BFC000360C26201F088F800B938BDBDE8384026
:100C0C00FFF7DEBF282300200030014038B5012259
:100C1C0000234FF4806502240D484FF40071C0E9A5
:100C2C000135C0E9033442610023002200240A2567
:100C3C00C0E90823074BC0E90A458161036001F054
:100C4C0063F800B938BDBDE83840FFF7B9BF00BF45
:100C5C00802300200038004070B500243D4A036812
:100C6C0088B093420546CDE90444CDE9064404D04E
:100C7C00394A934233D008B070BD384B04A99A69F5
:100C8C00374E42F480529A619A6902F48052009273
:100C9C00009A9A6942F004029A619B69A02203F0BF
:100CAC000403019301980320022307902D48CDE9FA
:100CBC00042300F04BFB80231022F3602A4B3046B8
:100CCC00C6E90444C6E90644B4607260336000F0BF
:100CDC00C1F9002838D1AE64756208B070BD1F4BE5
:100CEC002248DA6904A942F48042DA61DA69204EBA
:100CFC0002F480420292029A9A6942F008029A61C6
:100D0C009B6903F0080303934FF42043039A049365
:100D1C0000F01CFB8023174A3046C6E90024C6E9C4
:100D2C000444C6E90644B460F36000F093F970B96A
:100D3C00002224201146EE64756200F027F924206D
:100D4C0000F062F908B070BDFFF73AFFC3E7FFF798
:100D5C0037FFEDE700300140003800400010024042
:100D6C00A02200200008014030000240000C01408D
:100D7C00E4220020440002400E4B82B09A690E49D6
:100D8C0042F001029A619A6902F001020092009A03
:100D9C00DA6942F08052DA61DB6903F08053019327
:100DAC00019B4B6823F0E06343F000734B6002B08F
:100DBC00704700BF0010024000000140FEE700BF7A
:100DCC00FEE700BFFEE700BFFEE700BFFEE700BF87
:100DDC00704700BF704700BF704700BF00F0A0B85D
:100DEC00014800F01FBA00BFA0220020014800F00B
:100DFC0019BA00BFE4220020014801F049BB00BF32
:100E0C008023002008B5134B1B782BB9BDE8084094
:100E1C004FF4006000F0B8BB0F4801F0CFF90E485A
:100E2C0001F036F90D4B0C481A6942F480421A61F4
:100E3C001A6922F480421A6100F066FFEB2208491D
:100E4C00054801F0ADF8BDE808404FF4006000F033
:100E5C009BBB00BF34000020802300200010024008
:100E6C00B4010020704700BF0C480D490D4A002307
:100E7C0002E0D458C4500433C4188C42F9D30A4A43
:100E8C000A4C002301E013600432A242FBD3FFF7AB
:100E9C00E9FF01F085FBFFF769FD704700000020BA
:100EAC0014000020E829000818000020DC23002092
:100EBC00FEE7000038B54FF47A730D4A05461178F9
:100ECC000C4AB3FBF1F31268B2FBF3F000F0AAF892
:100EDC0008B90F2D01D9012038BD04460246294618
:100EEC004FF0FF3000F052F8034B20461D6038BD28
:100EFC000C0000200800002010000020074A08B554
:100F0C001368032043F01003136000F02DF80F203A
:100F1C00FFF7D0FFFFF730FF002008BD0020024094
:100F2C00034A044B11681B780B441360704700BFD5
:100F3C00D82300200C000020014B1868704700BF1C
:100F4C00D823002038B50446FFF7F6FF631C05468E
:100F5C0002D0044B1B781C44FFF7EEFF401BA04251
:100F6C00FAD338BD0C0000204FF6FF0C06490302E3
:100F7C00CA6803F4E06302EA0C02134343F0BF6354
:100F8C0043F40033CB60704700ED00E01C4B00B520
:100F9C00DB68C3F30223C3F1070EBEF1040F03F1A8
:100FAC00040C28BF4FF0040EBCF1060F1BD94FF0F8
:100FBC00FF3C033B0CFA03FC22EA0C024FF0FF3C13
:100FCC000CFA0EFC21EA0C019940002841EA0201BE
:100FDC000CDB090100F16040C9B200F5614080F8FA
:100FEC0000135DF804FB00221346E7E7054B00F005
:100FFC000F000901C9B2034419765DF804FB00BF68
:10100C0000ED00E0FCEC00E0002807DB012300F021
:10101C001F01034A40098B4042F82030704700BF43
:10102C0000E100E00138B0F1807F0FD24FF0E023F7
:10103C004FF0F00C0022072110B4054C586184F8D5
:10104C0023C010469A6110BC19617047012070478B
:10105C0000ED00E040B3034605C84FF4807C30B48B
:10106C0000249968DD680A4310492A43104D014455
:10107C00A5FB015109098900196419699D690A4385
:10108C0059690A4301682A43DD6921F47F5121F033
:10109C0030012A430A430749D9630260A3F820C0F0
:1010AC0020469C6330BC704701207047F8FFFDBFA1
:1010BC00CDCCCCCC00000240844690F82000012816
:1010CC003FD030B401249CF821008CF82040A04281
:1010DC0005D000238CF82030022030BC704702244D
:1010EC008CF821400024DCF84050CCF83840DCF877
:1010FC000040A840256825F001052560DCF83C502F
:10110C0068606360DCF80430102BDCF82C300BBF0B
:10111C00A260A160E160E26053B1236843F00E036A
:10112C0023602368002043F00103236030BC704728
:10113C00236823F004032360236843F00A0323602D
:10114C00EFE70220704700BF90F821200346022AE7
:10115C0006D004229A630022012083F820207047D5
:10116C004FF0010C1A680020116821F00E0111607B
:10117C00116821F001011160D3E90F120CFA02F28F
:10118C004A60002283F821C083F82020704700BFFA
:10119C0090F821200346022A03D0042201209A63EE
:1011AC007047026810B511681B4821F00E011160E0
:1011BC001168824221F00101116021D017498A4245
:1011CC001AD014318A421DD014318A421DD01431E8
:1011DC008A421DD014318A420CBF4FF480124FF05A
:1011EC0080724FF480700E4C596B6260188429B178
:1011FC0018468847002010BD1022F2E7084610BDA3
:10120C000122EEE74FF48072EBE74FF48052E8E7EF
:10121C004FF48032E5E700BF080002401C0002409A
:10122C0000000240042270B4C66B016C3468036881
:10123C008A4022421D681FD06A071DD51A68910684
:10124C0003D41A6822F004021A603E4A93425AD020
:10125C00143293425FD01432934266D014329342CC
:10126C0069D0143293425BD0143293420CBF4FF4CA
:10127C0080024FF0806247E002228A40224222D054
:10128C00AA0720D51A68910606D401211A6822F003
:10129C000A021A6080F821102A4A934229D014328B
:1012AC00934240D01432934242D01432934234D001
:1012BC001432934242D0143293420CBF4FF40012BA
:1012CC004FF0007216E008228A40224219D02A07F9
:1012DC0017D51A684FF4807422F00E021A6001239D
:1012EC00026B03FA01F17160836304844AB170BC30
:1012FC00104702220021144C836A626080F820108F
:10130C003BB970BC704704220F49C36A4A60002B7A
:10131C00F7D070BC18474022F6E74FF40052E9E7CB
:10132C004FF48022F0E72022E4E74FF48062EBE7F1
:10133C004FF40072DEE74FF48042E5E74FF40032E1
:10134C00D8E700BF08000240000002402DE9F04F32
:10135C000E6883B0002E00F0B58000227A4F9246C2
:10136C0013467A4DDFF8E88106E0013336FA03F4D0
:10137C0002F1040200F0A68001249C4034EA060E1F
:10138C0004EA060CF1D14E68122E00F29E80122E49
:10139C001AD8DFE806F0A7B9B5CE19191919191919
:1013AC0019191919191919B1BC00DFF8A8E17645FA
:1013BC0000F098800EF5702E764500F09380AEF517
:1013CC00801E764500F08E80BCF1FF0F9CBF8646D8
:1013DC0093464FF00F0684BF00F1040EA2F1200BD0
:1013EC00DEF800400AFA0BF906FA0BFB24EA0B04B0
:1013FC0044EA0904CEF800404C6814F0805F79D0C0
:10140C00D7F818E003F003094EF0010EC7F818E006
:10141C00D7F818E04FEA89090EF0010ECDF804E078
:10142C00DDF804E023F0030E0EF1804E0EF5803E45
:10143C00DEF808B006FA09F62BEA0606DFF818B152
:10144C00584513D00BF5806B58456BD0DFF80CB1B9
:10145C00584560D0DFF808B158450CBF4FF0030B6E
:10146C004FF0040B0BFA09F946EA0906CEF80860AE
:10147C002E6814F4803F14BF46EA0C0626EA0C06CC
:10148C002E606E6814F4003F14BF46EA0C0626EA80
:10149C000C066E60AE6814F4801F14BF46EA0C068E
:1014AC0026EA0C06AE6014F4001FEC681FD044EA68
:1014BC000C04EC600E68013336FA03F402F10402FA
:1014CC007FF45AAF03B0BDE8F08F46450AD07FF6E3
:1014DC006CAFDFF890E0764504D00EF5803E764593
:1014EC007FF472AF8E683EBB4FF0040A6CE724EABF
:1014FC000C04EC600E6838E7CC6804F1040A63E76E
:10150C00CC6804F1080A5FE7D1F80CA05CE7CC6862
:10151C0004F10C0A58E74FF0020B0BFA09F946EAF2
:10152C000906A3E74FF0010B0BFA09F946EA090685
:10153C009CE74FF0000A47E7012E4FF0080A0CBF5A
:10154C000461446140E700BF001002400004014008
:10155C000000221000001210000801400010014091
:10156C00001401400000311002B9090401617047F8
:10157C00C36801EA030221EA030141EA0241016165
:10158C00704700BF704700BF044A5169014200D147
:10159C00704708B55061FFF7F5FF08BD0004014026
:1015AC00002800F0B6812DE9F04103680446DD0700
:1015BC0082B035D59A494A6802F00C02042A00F030
:1015CC00EF804A6802F00C02082A00F0E58063689C
:1015DC00B3F5803F10D0002B00F00C81B3F5A02F99
:1015EC0000F082818E4B1A6822F480321A601A68DD
:1015FC0022F480221A6004E0894A136843F4803391
:10160C001360FFF799FC864E054605E0FFF794FC46
:10161C00401B642800F2EA8033689A03F6D52368ED
:10162C009F0728D57E4A516811F00C0F00F08D8071
:10163C00516801F00C01082900F083802369002B0C
:10164C0000F018810122774B754E1A60FFF774FC7D
:10165C00054605E0FFF770FC401B022800F2C6802F
:10166C0033689807F6D53368626923F0F80343EAC8
:10167C00C203336023681A071FD45D0742D5684B39
:10168C00DA69D0007DD50025674E3368D90540F165
:10169C009D80E368012B00F0FE80002B00F0CA80D7
:1016AC00052B5F4B1A6A00F02C8122F001021A62A2
:1016BC001A6A22F004021A62F2E0A369002B4FD0DE
:1016CC000122584B564EC3F88024FFF735FC0546D3
:1016DC0005E0FFF731FC401B022800F28780736A9B
:1016EC009B07F6D5514B524A1B68A2FB03235B0A9E
:1016FC00019300BF019B5A1E0192002BF9D1236864
:10170C005D07BCD4E069C0B1454D6B6803F00C03B8
:10171C00082B00F0D8800022424B02281A6600F0F9
:10172C00FA80FFF709FC044604E0FFF705FC001BF8
:10173C0002285BD82B689B01F7D4002002B0BDE8CF
:10174C00F0815268D6033FF579AF354A1268950798
:10175C0030D52269012A2DD0012002B0BDE8F081DC
:10176C00304A2F4EC2F88034FFF7E6FB054604E002
:10177C00FFF7E2FB401B022838D8736A9F07F7D4A7
:10178C00BDE7DA69012542F08052DA61DB6903F0CA
:10179C0080530093009B77E74A68D0037FF517AF1F
:1017AC001F4A126891037FF53BAF6268002A7FF4F1
:1017BC0037AFD1E71A4960690A6822F0F80242EAA9
:1017CC00C0020A601A077FF558AF76E7336843F416
:1017DC0080733360FFF7B0FB07463368DA053FF5DB
:1017EC0058AFFFF7A9FBC01B6428F6D9032002B041
:1017FC00BDE8F0810A4D2B6823F480332B602B68F5
:10180C0023F480232B60FFF797FB064604E0FFF7D9
:10181C0093FB801B6428E9D82B689B03F7D4FEE666
:10182C0000100240000042420070004008000020FE
:10183C00D34D6210504E41F28838336A23F00103C5
:10184C003362336A23F004033362FFF775FB0746F8
:10185C0004E0FFF771FBC01B4045C7D8336A9807FB
:10186C00F7D4002D3FF44EAF434AD36923F0805395
:10187C00D36147E7414A404E1360FFF75DFB0546D5
:10188C0004E0FFF759FB401B0228AFD833689907D7
:10189C00F7D42368EFE6384A136A43F00103136266
:1018AC00FFF74AFB41F288380646334F04E0FFF756
:1018BC0043FB801B404599D83B6A9B07F7D5002D0D
:1018CC003FF420AFD0E701283FF438AF6B68226AB1
:1018DC0003F4803191427FF43FAF606A03F47013DC
:1018EC00181A18BF012029E703F18043A3F53C33F4
:1018FC001A6842F480221A601A6842F480321A6024
:10190C007FE642F004021A621A6A42F001021A627D
:10191C00C6E701207047FFF70FFB064605E0FFF70F
:10192C000BFB801B02283FF661AF2B689901F6D4A4
:10193C00236AB3F5803F05D16A68A16822F40032AE
:10194C000A436A6001200C4D616A6A680B4322F4F9
:10195C0074120A4913436B600866FFF7EDFA0446EC
:10196C0005E0FFF7E9FA001B02283FF63FAF2B68B2
:10197C009A01F6D5E1E600BF001002400000424299
:10198C00002800F0B1805E4A2DE9F041136804464E
:10199C0003F007038B420D4686B00DD2136823F07B
:1019AC0007030B431360136803F007038B4203D048
:1019BC00012006B0BDE8F08123689E0714D55807B6
:1019CC0004D550494A6842F4E0624A60190704D5CC
:1019DC004C494A6842F460524A604A49A0684A68D5
:1019EC0022F0F00202434A60DA0720D56268454BC8
:1019FC00012A1B687AD0022A73D09E07D8D5414E93
:101A0C0041F28838736823F0030313437360FFF7C4
:101A1C0093FA074604E0FFF78FFAC01B404568D8DD
:101A2C007368626803F00C03B3EB820FF3D1344A92
:101A3C00136803F00703AB4209D9136823F00703BB
:101A4C002B431360136803F00703AB42B0D1236838
:101A5C00580706D52B49E0684A6822F4E062024335
:101A6C004A60190707D5274A2169536823F4605344
:101A7C0043EAC103536040F20124234B06AD0FCB64
:101A8C0005E90F001F49ADF804404A6802F00C0349
:101A9C00082B11D01D4B1B4A1D4852681D49C2F31F
:101AAC000312805C1C4AC34008681360FFF702FAFB
:101ABC00002006B0BDE8F081C2F3834318336B44B9
:101ACC00D20313F8103C16D54A681049C2F34042B1
:101ADC0001FB03F318326A4412F8142CB3FBF2F333
:101AEC00D9E79F018BD463E7012070479B0386D411
:101AFC005EE703205DE7094A02FB03F3CBE700BF77
:101B0C000020024000100240CC29000800127A008C
:101B1C00BC290008100000200800002000093D002E
:101B2C004FF0640C0021154B154A1B6882B0A2FBC8
:101B3C0003235B0A0CFB03F300910268019305E09D
:101B4C00019B013B019393689B0706D4019B002BDF
:101B5C00F6D1436D43F0400343650721136823F02E
:101B6C0040031360536823F0E0035360D368009381
:101B7C00009B80F8511002B0704700BF0800002095
:101B8C00F1197605072103685A6822F080025A6021
:101B9C001A6822F040021A6080F85110704700BF9A
:101BAC002DE9F0411D46164682B00C460746FFF75C
:101BBC00C3F935442D1AFFF7BFF98046264B1B6835
:101BCC00C3F3CB3305FB03F30193731C396807D1C3
:101BDC008B6834EA0303FBD0002002B0BDE8F0812F
:101BEC008B6834EA0303F7D1FFF7A6F9A0EB0800E2
:101BFC00A84207D2019B002B019B08BF0025013B8B
:101C0C000193E2E7D7E900315A68B1F5827F22F0FF
:101C1C00E0025A6013D0BA6AB2F5005F07D11A68B5
:101C2C0022F400521A601A6842F400521A6001221F
:101C3C000023032087F8512087F85030CDE7BA688D
:101C4C00B2F5004F02D0B2F5806FE4D11A6822F0E1
:101C5C0040021A60DFE700BF0800002070B50C4698
:101C6C0082B00646FFF768F96434241AFFF764F96A
:101C7C00244B32681B68C3F3CB3304FB03F301938F
:101C8C0093681A062FD505460AE0019A019B316824
:101C9C00013B01938B68002A08BF00241B0622D548
:101CAC00FFF74AF9401BA042EFD3D6E900315A683E
:101CBC00B1F5827F22F0E0025A6017D0B26AB2F519
:101CCC00005F07D11A6822F400521A601A6842F4B5
:101CDC0000521A6001220023032086F8512086F856
:101CEC00503002B070BD002002B070BDB268B2F5C9
:101CFC00004F02D0B2F5806FE0D11A6822F040029A
:101D0C001A60DBE708000020002858D0F8B5436AB9
:101D1C000446002B44D00023C0E90433002094F87F
:101D2C005130A06203F0FF02002B3FD0D4E9013206
:101D3C0002264FF0010C002502F4044203F48273D6
:101D4C001343E26884F85160266902F4006213437D
:101D5C0006F0020633436669A169276A06EA0C0697
:101D6C003343E66907F0800E01F4007706F038067D
:101D7C003B432268334343EA0E0303431068090CC8
:101D8C0001F0040120F04000106013605160D36931
:101D9C00284623F40063D361656584F851C0F8BD0F
:101DAC004268B2F5827FB9D0C361B7E7204684F8A8
:101DBC005020FEF751FFA06A00F40050B6E7012056
:101DCC00704700BF70B590F85030012B56D00446C8
:101DDC00012094F8513084F850008342DDB205D0D4
:101DEC000225002384F85030284670BD0029F8D015
:101DFC00002AF6D000230326A06884F85160B0F5C1
:101E0C00004F6365A286E286C4E910332268216321
:101E1C00A363A387E38728D00023A06C194E4363E8
:101E2C00E38EC662184E0C328662184E9BB2066365
:101E3C00FFF742F988B923681A68520603D41A6866
:101E4C0042F040021A605A68002542F020025A60A3
:101E5C005A6842F002025A60C3E70122636D43F0F4
:101E6C001003636584F85120BBE7136823F040032B
:101E7C001360136843F480431360CDE702252846B2
:101E8C0070BD00BF192200086D220008492200080D
:101E9C0038B5044690F8500001286CD04FF0010C76
:101EAC0094F85100656860455FFA80FE84F850C074
:101EBC000DD0B5F5827F04D00220002384F8503079
:101ECC0038BDA0680028F7D1BEF1040FF4D1002969
:101EDC004FD0002A4DD0002B4BD094F85100002548
:101EEC0004281CBF052084F8510000206065E3869F
:101EFC00E387A386A38794F851302163042BC4E9AC
:101F0C00100008BF2149E06C0EBF214B2149224B28
:101F1C00A263C0E90A312149E38F016321689BB2B6
:101F2C000C314563FFF7C8F8014630BB2268A06C42
:101F3C0053680C3243F0010342F8083CE38EC0E9CD
:101F4C000A11C0E90C119BB2216BFFF7B5F8A0B9CF
:101F5C0023681A68520603D41A6842F040021A60C9
:101F6C005A6842F020025A605A6842F002025A60E3
:101F7C00A3E70120A1E7022038BD0122636D1046C2
:101F8C0043F01003636584F8512096E7292200087A
:101F9C00E9220008392200083924000849220008E7
:101FAC002DE9F041856804460E461DB94368B3F52A
:101FBC00827F59D094F85030012B5ED0012194F8D7
:101FCC00513084F850108B42DFB206D00227002328
:101FDC0084F850303846BDE8F081002EF7D0002A46
:101FEC00F5D000230421B5F5004F84F85110A663F9
:101FFC0063652168E287A28723646364A386E38612
:10200C0029D00023E06C1F4D4363E38FC5621E4D46
:10201C00324685621D4D0C319BB20563FFF74CF8BF
:10202C0088B923681A68520603D41A6842F0400231
:10203C001A605A68002742F020025A605A6842F02F
:10204C0001025A60C3E70122636D43F0100363651C
:10205C0084F85120BBE70B6823F040030B600B683E
:10206C0023F480430B60CCE7042580F851501346D1
:10207C00BDE8F0410A46FFF70BBF02273846BDE822
:10208C00F08100BF29220008E9220008492200083B
:10209C006421464B464A1B6810B5A2FB03235B0A1E
:1020AC0001FB03F384B00293029B02680193536813
:1020BC00044623F0200353605368190613D53D4B97
:1020CC004364019B4BB1019B013B019394F851304C
:1020DC00072B06D0019B002BF5D1636D43F0400319
:1020EC006365029B019353685B0612D5324B2364E4
:1020FC0006E0019B013B019394F85130072B06D06D
:10210C00019B002BF5D1636D43F040036365029B8B
:10211C000193536898071AD5A06CC0B10023436390
:10212C00FFF712F800283DD12268536823F0020310
:10213C00536005E0019B013B01939368990706D41A
:10214C00019B002BF6D1636D43F04003636553682C
:10215C00DB0711D5E06C78B100234363FEF7F4FF85
:10216C0008B1402363652268136823F040031360B1
:10217C00536823F0010353600023E387E386616D0A
:10218C0040294FF000011ABF636518460120012356
:10219C000391D168039192680392039A84F85130A9
:1021AC0004B010BD40236365BEE700BF08000020EB
:1021BC00F1197605911B00082D1B000838B5044653
:1021CC00806C10B1FEF7C0FFA0B90025E06C38B1EF
:1021DC00FEF7BAFF20B10125636D43F01003636570
:1021EC00012122682846536823F00303536084F8C6
:1021FC00511038BD636D012543F010036365E5E7AD
:10220C00704700BF704700BF704700BF08B5406AF9
:10221C00FFF7FAFF08BD00BF704700BF08B5406A62
:10222C00FFF7FAFF08BD00BF704700BF08B5406A52
:10223C00FFF7FAFF08BD00BF704700BF0121406ADD
:10224C0008B50268536823F003035360436D43F0F1
:10225C001003436580F85110FFF7EEFF08BD00BF77
:10226C0030B5054683B0446AFEF766FE2B681B68E2
:10227C009B061DD4236801465A68204622F0200292
:10228C005A605A6822F002025A60FFF7E7FCA0B9C4
:10229C00A36833B922680193D368019393680193BF
:1022AC00019B01230022E28684F85130636D83B9CF
:1022BC002046FEF737FA03B030BD636D43F02003C0
:1022CC006365636D43F020036365A368002BE8D15D
:1022DC00E0E72046FFF7B0FF03B030BD70B506460F
:1022EC0082B0456AFEF728FE33681A68910653D40B
:1022FC002968AB684A68044622F020024A60002B29
:10230C004FD068684A68B0F5827F22F001024A60BB
:10231C006AD0FEF711FE6434241AFEF70DFE424B10
:10232C002A681B680646C3F3CB3304FB03F3019303
:10233C0093681B060BD428E0019A019B2968013B8A
:10234C0001938B68002A08BF00241A061DD5FEF7DE
:10235C00F3FD801B8442EFD8D5E900315A68B1F502
:10236C00827F22F0E0025A6032D0AA6AB2F5005F96
:10237C0025D00123002285F851306B6D85F8502053
:10238C0043F020036B6520236B6501230022EA8751
:10239C0085F851306B6D6BB92846FFF731FF02B0F1
:1023AC0070BD6B68B3F5827F4B6825D023F00103B9
:1023BC004B60AEE72846FFF73FFF02B070BD1A68CE
:1023CC0022F400521A601A6842F400521A60D0E7E4
:1023DC00AA68B2F5004F02D0B2F5806FC5D11A6869
:1023EC0022F040021A60C0E7B3F5004F08D10B6829
:1023FC0023F040030B608CE723F003034B6088E76A
:10240C00B3F5806F85D10868234620F04000086042
:10241C00642201212846FFF7C3FB0028B5D06B6D61
:10242C0043F020036B65AEE70800002038B5054685
:10243C00446AFEF781FD2B681B689B0616D4226844
:10244C0001465368204623F020035360FFF706FC37
:10245C0080B90022012021684B6823F003034B60F4
:10246C00E286E28784F85100636D63B92046FFF77A
:10247C00C9FE38BD636D43F020036365636D43F0A3
:10248C0020036365E5E72046FFF7D6FE38BD00BFA5
:10249C00026810B551689368044603F0410CBCF116
:1024AC00010F84B04FD0980701D5080653D413F010
:1024BC00600F46D0880644D558060ED594F85100C6
:1024CC00032852D0606D40F004006065002001903C
:1024DC00D068019090680190019898060CD5002066
:1024EC00636D43F001036365039093680393136872
:1024FC0023F040031360039B636D13B301205368F7
:10250C0023F0E00353608B0784F8510029D0536803
:10251C00E06C23F00303536040B1184B4363FEF7A8
:10252C0037FE18B1636D43F040036365A06C40B196
:10253C00124B4363FEF72CFE18B1636D43F040035E
:10254C00636504B010BD11F0400FACD0036C04B047
:10255C00BDE8104018472046636C04B0BDE810403D
:10256C0018472046FFF768FEEBE700230293D36879
:10257C00029393680293029BE3E700BF8D2500084A
:10258C0008B50023406AC387C386FFF755FE08BD14
:10259C0003460244934200D1704703F8011BF9E74C
:1025AC0070B500260C4D0D4C641BA410A64209D12D
:1025BC0000F01AF800260A4D0A4C641BA410A6421F
:1025CC0005D170BD55F8043B98470136EEE755F838
:1025DC00043B98470136F2E7E0290008E02900089F
:1025EC00E0290008E4290008F8B500BFF8BC08BCD5
:1025FC009E467047F8B500BFF8BC08BC9E467047B5
:10260C000807060504030201001213141516171807
:10261C00191A1B1C1D1E1F2021222311100F0E0D19
:10262C000C0B0A092E2D2C2B2A29282726252400B1
:10263C00000000F0F0F0000000F0FFF00F00000FC1
:10264C0000F0F0FFF0F000F000F00FFF00F00F0FC3
:10265C000F0F00F0000FFF00FFF000F000F00F0074
:10266C00FFF0000FF000FFFF000FFF0FF00FF00066
:10267C000F0F00F0FFF0F000FF0FF000F000FF0074
:10268C00FF00F00FF00FFF0F00F0FFF00F00F00055
:10269C0000FFF00FF00FFF0F000F00FFF0F00F0F17
:1026AC000000F0FFF0F00F000FFF0FF00FFF000025
:1026BC000000000FFF00000000F0F00F0F0000F012
:1026CC00F0F0F00F0F0F00F00F0F0F0F00FF0F0FB8
:1026DC000F0F00F0000F00F0F00000FF0FF0F0F013
:1026EC000F0000F00F00000F000F000F0F0F0F0076
:1026FC000F0FF0F0F00F0F00F00F0F0F0F00F0F0B6
:10270C00F00F0F0F0F0F000F0F0F0F000F0F0F0019
:10271C000F00000F0F0F000FF0FF000F00F00F0F56
:10272C000000F00F00FF0F000F000F0F0F0F000045
:10273C0000000FFF0FFF000000F0F00F0F0000FF74
:10274C00F0F0F00F0F0F00F00F0F0FFF00F0FF0F66
:10275C000F0F00F0000F00F0FF0000F0F0F0FFF0A2
:10276C000F0000FFFF0000F0000FF00F0F0F0F0025
:10277C000F0F0FF0FF0F0F00FF0F0F0F0F00F0F0F8
:10278C00FF0FFF0F0F0FFF0F0F0F0F000F0F0F0F8C
:10279C000F0FF00F0F0FF00F0F0F000F00F00FF0D7
:1027AC000000F00F00F0FF000FFF0F0F0F0F0000E5
:1027BC000000000FFF00000000F0F00F0F0000F011
:1027CC00F0F0F00F0F0F00F00F0F0F0000F00F0FD5
:1027DC000F0F00F0000F00F0F00000F000F0F0F030
:1027EC000F0000F00F000F00000F000FF00FF000B3
:1027FC000F0F00F0F00F0F00F00FF00F0F00FF00A5
:10280C00F00F0F0FF0000F0F0F0F0F000F0F0F0037
:10281C000F00F00FF00F000F000F000F00F00F0F64
:10282C000000F00F00F00F00000F0FF00F0F000072
:10283C00000000F0F0F0000000F0FFF00FFF00F0DF
:10284C00F0FFF00F00F000FFF0F00F0000F00F0FA2
:10285C00FF0FF0FF000FFF00F00000F000F0F0F0B1
:10286C000F0000F00F00FFFF000FFF0F0F0F0F0006
:10287C000F0F00F0F000F000F00F0F00F000F0F080
:10288C00FF0F0F0F0F0FFF0FF0F00F000FF0F00006
:10289C0000FFF00F0F0FFF0F000F000F00FF0F0FC7
:1028AC000000FF0F00F00F000FFF0F0F0FF0F000F4
:1028BC00000000000000000000FF000000FF00000E
:1028CC000000FFFF0000FF00000000FF00FF000001
:1028DC00FFFF000000FFFFFF00FF00000000FF00F3
:1028EC0000FF00FF00FF0000FF00FFFF00FFFF00E4
:1028FC000000FFFF00FF00FFFFFF0000FFFFFFFFD6
:10290C00FF00000000FF000000FFFF0000FF00FFC1
:10291C000000FFFFFF00FF0000FF00FF00FFFF00B3
:10292C00FFFF00FF00FFFFFFFFFF000000FFFF00A5
:10293C0000FFFFFF00FF00FFFF00FFFFFFFFFF0096
:10294C0000FFFFFF00FFFFFFFFFF00FFFFFFFFFF88
:10295C000000000000F0000F00000FF000F000007D
:10296C00F0F000FF0000FFF00F00000F00F00F0F61
:10297C00000F0FF00FF0000FF0F00FFF000FFFF043
:10298C00F00000F000F0F00F00F00FF0F0F000F0AD
:10299C00F0F0F0FF00F0FFF0FF0000FF00F0FF0F81
:1029AC0000FF0FF0FFF000FFF0F0FFFF00FFFFF063
:1029BC0000000000000000000102030406070809E3
:1029CC0002030405060708090A0B0C0D0E0F101064
:0429DC0000000000F7
:0429E00031010008B9
:0429E4000D010008D9
:1029E80040000001010000000024F4000100000084
:0429F80010000000CB
:0400000508000E756C
:00000001FF
